:020000005D2879
:1000080009008A01033982070834023400340A34AB
:100018008A010339820720340434003424348A01E5
:100028000339820747344F3457345F348A013F39E4
:1000380082070034013402340334043405340634AE
:1000480007340134003403340234053404340734EB
:1000580006340234033400340134063407340434DB
:1000680005340334023401340034073406340534CB
:1000780004340434053406340734003401340234BB
:1000880003340534043407340634013400340334AB
:10009800023406340734043405340234033400349B
:1000A800013407340634053404340334023401348B
:1000B800003483161F308500003086000E309F0004
:1000C80070308F0083120030920000308600850067
:1000D800B501B60106102921A611B1013108252163
:1000E80050309321061234213421261C94280616F8
:1000F800A61D8628A6113C30A700EC20A61990283A
:10010800A70B8128EE2031081320A2201E3093214E
:1001180030080A3C031894289B20463093219528E0
:100128000612B10A3108043A031D722871283108F1
:10013800B200272131081320CB200800B3003F303C
:10014800B400AF01B001AF030830B9003308840030
:100158000008B700340884000008B7023708B71B46
:10016800003CA800BC20B30AB40AB90BAA280800AE
:1001780028082F020318C52828083002031CC8289D
:1001880008002808AF0008002808B0000800B400DC
:100198003F30B300CF280830B90033088400000886
:1001A800B7003408840037088000B30AB40AB90BD2
:1001B800D12808002611B700B71B003C0A3C031CD5
:1001C800261508001430A700EC20A70BE828080023
:1001D800783093290B21BD011E3058210830BB000F
:1001E8000C30BE000830BC000F30582101305821B7
:1001F8003E085421851468218510A8001E21BD0AD7
:100208000A30BE07BC0BFA28BB0BF42808003F30A5
:1002180084000830B9008001840AB90B0F2908004E
:100228003F3084000830B90000086F21840AB90BF8
:10023800182908003D0807393F3E84002808800730
:100248000800B6002929B500292936080520B70075
:1002580035080C20B7040608D13937048600080091
:1002680026100630B9004121A61808000F3C0318D3
:100278003429B90B372926140800A6146430B800AD
:10028800051A4929B80B442908006430B800051E2E
:100298005029B80B4B2908003808643CA610080000
:1002A800B700B70B55290800B700B801051E5F292C
:1002B800B80B5A290800B801051A6529B80B602936
:1002C8000800B70B59290800370885309F001F1907
:1002D8006B291E080800A0000830A10086178A2193
:1002E8008A2186138A2186178A21201C86138A214F
:1002F80086138A21A00CA10B772986178A218613D9
:100308001E30A1008A21A10B862908001430A20002
:100318000000000000000000A20B8C290800A500C6
:10032800A400851CA615A300A30B9829A40B972944
:06033800A50B942908004A
:02400E00222F5F
:00000001FF
